:10000000370101002920A9487300000082804EB802
:10001000130101801301018805650A95233485FACF
:1000200028009305F57F9385157A23200500110597
:10003000E31DB5FE2245B245130685003365A520B4
:100040002E9513058504B3F5C50E3355C50EB3E4DF
:10005000A50013F5F40FC1201385D401619D652817
:1000600013844402619C22857D2022856D201385A6
:100070007402619D4D204245D2451306450033650B
:10008000B52013050502B3F5C50E3355C50E33E48F
:10009000A5001375F40F41206245930555003346C2
:1000A000A5203325A6202295130575033376B40EBB
:1000B0003355B50E3364A6001375F40FA928130544
:1000C0008401619D89281305B401619DA920130550
:1000D0005401619D89201305D400619D2D2803459D
:1000E000C10113051502619D3D200345010229054B
:1000F000619D85658A9503B485FA1301017F13011B
:1001000001794EBA09A885487300000082809148A1
:10011000730000008280AD48730000008280930865
:1001200010087300000082809308500873000000DC
:10013000828093087008730000008280732510C0CD
:100140008280732500C082809308600873000000DD
:1001500082800589F322008093920248B3E2A200D4
:10016000739002808280954873000000828093081B
:100170000008730000008280A148730000008280A4
:1001800093083008730000008280930840087300D1
:040190000000828069
:00000001FF
